:1000000011298030A100FE30AF200130AF207530C3
:10001000A7003030C628A101A117AF00AF08031D0B
:100020001328030114280130AF020310A20CA20C04
:10003000A20CC0302205403EAF07FE30AF202F0893
:10004000AF28A101A117AF00FE30AF202F08AF28C5
:10005000A401AA00AB01A01124080319A0150530C2
:10006000A3002730A900103041200330A900E83058
:100070004120A90164304120A9010A3041202A0809
:100080004828A8002B08A7002A08A600DA2026087E
:10009000A600A3030319A011240803195228230260
:1000A000031859282608031DA011A0195928303E0D
:1000B000AF280800A300240803190C292308AF2047
:1000C000A4035B28AD000611861183160611861164
:1000D0000F30860583122D08A0188C283E30A7000B
:1000E0008030C6203330AC00A0201330A700883009
:1000F000C620A0206430C520A0206430C520223056
:10010000AC00A02028308B200C308B2006308B20B8
:10011000A0142D088C282014AC00201C9A288611CD
:10012000033C031C9F289F200530A700DC30C6201D
:10013000031408002014FE3C0319AD288615201C6A
:10014000201006150F3086052C08F039860406119C
:10015000AC0E2018A0283230C5202D080C29A11B78
:10016000622883178001840AFF3E031DB2280C29F0
:10017000A901A800FF30A807031CA907031C0C292C
:100180000330A700DF30C620BA28A701E83EA6004A
:10019000A709FC30031CCF28A6070318CC28A60704
:1001A0000000A70FCC282618D528A61CD9280000A7
:1001B000D9280800AB01AA011030AC00270DAA0D08
:1001C000AB0D2808AA022908031C290FAB0203184B
:1001D000F0282808AA0729080318290FAB070310DD
:1001E000A60DA70DAC0BDE2826080C291030B00098
:1001F000A701A601AD0CAC0C031C04292808A60716
:1002000029080318290FA707A70CA60CAB0CAA0CEA
:10021000B00BFA282A080C29831383120313000059
:100220000800A00107309F00E03083168500FF30F2
:10023000860081138312850186012030840060309E
:10024000B220A03084005030B22020308400303002
:10025000B120C830B82001207730622062206220AF
:100260002E3062207030622069306220633062205C
:100270006230622061306220733062206930622017
:10028000633062202E3062206E3062206C3062203B
:100290000B30A900B830B92001204430622043302F
:1002A0006220463062203130622036306220553084
:1002B00062204B3062204330622020306220622076
:1002C000563062202D306220323062200730A90083
:1002D000D030B920012041306220643062206A3081
:1002E00062207530622073306220743062202030CA
:1002F00062204C30622044306220523062208618E6
:100300008729851F85290514862905107F29012045
:10031000533062206530622061306220723062208A
:1003200063306220683062202030622073306220A7
:1003300069306220673062206E3062206130622056
:100340006C30622036140512831605128312302A8F
:10035000C3013C03A500C90149082502031CC129AA
:10036000E421B61CBF294308A6004908A200A60143
:10037000A20A0314A60DA20BBA292608C304C90FAA
:10038000AC29B2014308B100B20CB10CB20CB10CF3
:10039000B20CB10CB20CB10C0F30B2053208AD008A
:1003A0003108AC00A9010A30A800F620B1002B08E2
:1003B000B200B4014308B3000F30B3050030B405F8
:1003C00031083307C3000800BA01B9010618F9293A
:1003D0000130B820B90A0319BA0A0B303A02031CDB
:1003E000F829031DF729B9303902031CF829542DC7
:1003F000E6299B30B8200618B614061CB610361C29
:100400001A2A440EB100B200F030B1050F30B20527
:100410003208A7003108A600A9013A30A800DA2066
:10042000BD008030A1000230A2003D080D20FF3049
:100430006220232A03013619013EB618013A031936
:100440003611031D3615C40A85140130A900F43095
:10045000B9208510A901F030A8002808B9200800AB
:10046000BB01C4013612361AC32ABA01B901061CEF
:100470004A2AB90A0319BA0A0130B820AF303A0241
:10048000031C492A031D482AC9303902031C492A82
:10049000542D372ABA01B90106187C2AB90A031962
:1004A000BA0A0A30B8203618702A39080B3A3A04CA
:1004B000031D5B2A6F2A3908193A3A04031D622A80
:1004C00085146F2A39084B3A3A04031D692A8510AE
:1004D0006F2A3908FA3A3A04031D6F2A542D7B2AF1
:1004E00011303A02031C7B2A031D7A2A9530390207
:1004F000031C7B2A542D4C2A41303B02031C812AC9
:10050000542DBB0A3A08031D892A65303902031CA1
:100510008A2A3616361CC22A3B0EB100B200F030D1
:10052000B1050F30B2053208A7003108A600A901B5
:100530004130A800DA20BD008030A10080302120A9
:10054000463062206F306220753062206E3062204B
:100550006430622020306220733062206930622073
:10056000673062206E306220613062206C30622021
:10057000203062208030A1000230A2003D080D2012
:10058000FF306220332A361CE72A012049306220DE
:100590006E306220693062207430622069306220DF
:1005A000613062206C306220693062207A306220D3
:1005B000653062202E306220622062208030A100EF
:1005C000C03021201030A4005F305A204C2B0B305B
:1005D000BD000130A2003D080B20A101B61DFF2A7D
:1005E0003B3041020318F62AC10AFE2AC101173026
:1005F00045020318FD2AC50AFE2AC501032B42083D
:10060000C1004608C500051B132B4508031D0B2B15
:100610000C30C700122B0D304502031C122B0C307E
:100620004502C700172B4508C700203062200A305A
:10063000470203181D2B203062208030A10047089C
:1006400028203A3062200230A40041082920051BEE
:10065000352B0C3045020318302B61306220322BD1
:10066000703062200E30BD00372B0F30BD004108C6
:1006700003190130031D0301B5001E3041020319A7
:100680000130031D03013504B50001308618030154
:10069000350403194C2B2C2D361E2A2DE421013054
:1006A000C9000F3049020318582BE421C90F512B00
:1006B0003611B611E421E421E421B61C612B0514A6
:1006C000622B05101230C9001430490203186B2B3D
:1006D000E421C90F642BE4210730BC00A8214308A2
:1006E000C200E421361D752BB6150630BC00A821CA
:1006F0004308C600E421361D7E2BB6150630BC002B
:10070000A8214308BE000330BC00A8214308C8004C
:100710000530BC00A8214308C0000830BC00A82157
:100720004308BF00E421361D962BB615361C9C2BC2
:10073000B6199B2B36100120B619292D8030A10047
:10074000803021200930A40020305A208030A100C0
:10075000C03021201030A40020305A2080302120C9
:10076000A10101304802031DC22B4D3062206F30C1
:1007700062206E3062206430622061306220793005
:100780006220372C02304802031DD52B54306220E2
:1007900075306220653062207330622064306220E0
:1007A0006130622079306220372C03304802031D0B
:1007B000EC2B5730622065306220643062206E304E
:1007C00062206530622073306220643062206130C4
:1007D000622079306220372C04304802031D012C3E
:1007E000543062206830622075306220723062209E
:1007F0007330622064306220613062207930622080
:10080000372C05304802031D122C4630622072300E
:100810006220693062206430622061306220793069
:100820006220372C06304802031D272C53306220EB
:100830006130622074306220753062207230622034
:10084000643062206130622079306220372C0730BA
:100850004802031D372C53306220753062206E3001
:100860006220643062206130622079306220803002
:10087000A100C03021203E08282020306220013015
:100880004002031D522C4A306220613062206E30DB
:1008900062207530622061306220723062207930CF
:1008A00062200E2D02304002031D672C463062206C
:1008B00065306220623062207230622075306220C2
:1008C0006130622072306220793062200E2D033058
:1008D0004002031D762C4D30622061306220723060
:1008E000622063306220683062200E2D04304002A6
:1008F000031D852C413062207030622072306220EE
:10090000693062206C3062200E2D05304002031DDC
:10091000902C4D30622061306220793062200E2DA3
:1009200006304002031D9D2C4A3062207530622043
:100930006E306220653062200E2D07304002031DAC
:10094000AA2C4A306220753062206C3062207930E7
:1009500062200E2D08304002031DBB2C4130622066
:1009600075306220673062207530622073306220FB
:10097000743062200E2D09304002031DD22C5330FA
:1009800062206530622070306220743062206530F1
:1009900062206D30622062306220653062207230E9
:1009A00062200E2D0A304002031DE52C4F306220DC
:1009B00063306220743062206F30622062306220C7
:1009C00065306220723062200E2D0B304002031D14
:1009D000FA2C4E3062206F30622076306220653013
:1009E00062206D3062206230622065306220723099
:1009F00062200E2D0C304002031D0E2D443062206B
:100A00006530622063306220653062206D30622084
:100A1000623062206530622072306220093040020C
:100A2000031D1D2D20306220273062208030A10060
:100A30000230A4003F082920292D203062203230C6
:100A40006220303062208030A1000230A4003F08D4
:100A500029202B2D542D302A851F332D0512831666
:100A600005128312352D8316051683129B30B8208C
:100A7000410803190130031D0301B5000130861838
:100A8000030135040319452D05158515851401301D
:100A9000A900F430B9200511851185100130A90095
:100AA0004A30B920C40A4F2B01204E3062206F30EB
:100AB000622020306220733062206930622067300B
:100AC00062206E306220613062206C306220203003
:100AD00084006030B220A03084005030B22020303A
:100AE00084003030B1200618B616061CB612030179
:100AF0000618013EB61A013C031D842DB70A0319DE
:100B0000B80A0130B820772D0301B61A0130013A36
:100B10000319B612031DB61603010618013EB61AD4
:100B2000013C031D992DB70A0319B80A0130B820FA
:100B30008C2D03303802DE30031937020318672D7D
:040B40003614302A0D
:02400E00503F21
:00000001FF
